:020000020000FC
:1000000020C109C039C067C085C085C085C086C011
:10001000F7C016C182C03F932F931F931FB71F9342
:1000200060FB2EF46E7F18B3137F18BB1FC012FB4A
:1000300096F4209173003091720011E0211B3F096A
:100040002093730030937200232B222321F418B3E2
:10005000137F18BB6B7F2091A1003091A00011E0AD
:10006000210F3F1D2093A1003093A0001F911FBFBF
:100070001F912F913F9118952F931F931FB71F9397
:1000800061FB2EF46D7F12B31F7C12BB1FC013FBEC
:1000900096F4209175003091740011E0211B3F0906
:1000A0002093750030937400232B222321F412B384
:1000B0001F7C12BB677F2091A3003091A20011E04A
:1000C000210F3F1D2093A3003093A2001F911FBF5B
:1000D0001F912F9118951F922F923F924F921F932D
:1000E0001FB71F9310907700209076003CB44DB45A
:1000F0003092770040927600311842083092A50085
:100100004092A4001F911FBF1F914F903F902F90CE
:100110001F90189518951895189518952F933F933B
:100120000F92AF93BF93EF93FF931F922F923F9243
:100130001F931FB71F9320E61BB114FB76F910FB2A
:100140002EF01CB1312E77FB36F011C01CB1312ED0
:100150001AB111FB66F010906F00112009F442C033
:1001600010906B0020906C00121834F132C0109186
:100170009F001F71232C269426942694211A31F077
:10018000F0926F00F0926B0078682CC07068777FF7
:100190001AE0109370001FEF10936F00F0926B0045
:1001A00017E03122E9E9F1E08894EE1FFF1FE30D2B
:1001B000FF1DC89500926C0030916B00230FBB2788
:1001C000A22F3C92339530936B001AE0109370008D
:1001D00009C030916B00230FBB27A22F3C921FEF69
:1001E00010936E001F911FBF1F913F902F901F9083
:1001F000FF91EF91BF91AF910F903F912F91189583
:10020000AF93BF931F931FB71F9310916D0013956A
:1002100010936D00155041F0A6E610916D00A10FEE
:10022000BB271C911CB906C053985598F0926800E2
:10023000F09269001F911FBF1F91BF91AF91189558
:1002400018951FED1DBFFF24A0E6B0E0FD9219ED4B
:100250001A1BE1F71FE015BF10EC1BBF18E019BF18
:1002600012E013BF10E01FBD11E01EBDA89518E0FD
:1002700011BD112718BB12BB1CEF17BB11E711BB37
:1002800014E11AB91CE019B913E018B92BD05CD1EC
:1002900092D1B5D17894DD24F2BE8CE792B798174D
:1002A000EAF31CE7810FE6E6F1E013E0D122ED2C42
:1002B0008894EE1C8894EE1FFF1FEE0DFF1DC8955D
:1002C000E6E6F1E0E00DFF1DD3940994040006007A
:1002D00008000A0032D0E2CF38D1E0CF6DD1DECFB6
:1002E0008FD1DCCF77276627FBBCFABC1FEF18BB8A
:1002F00012BB22E03327AEE9B0E01CB310FBEEF3F3
:100300003EBB11E01CBB1DB31D9333952A952223E0
:10031000A1F716B310FB70F90EF0529811FB2EF0F6
:1003200017E619B9F0929F00089510919E0019B92F
:100330000895010303010101030210906E001120D2
:1003400009F400C1F0926E00F0926800F09269002A
:10035000E9EBF1E0109060008894111C8894EE1F86
:10036000FF1FE10DFF1DC895E9EBF1E0E00DFF1D5A
:1003700009940800300054007E008A00980099001B
:10038000B7001091610010FB96F413FB6A7E60F9D0
:1003900011FB46F412FB1EF4C298C39AD2C0C29A53
:1003A000C39ACFC012FBDEF7C398C29ACAC013FB30
:1003B0006C7D61F911FB46F412FB1EF49498959A3A
:1003C000C0C0949A959ABDC012FBDEF79598949A96
:1003D000B8C020916200309163001091610010FB61
:1003E00076F420937200309373006E7E646011FB8C
:1003F0001EF4C298C39AA5C0C398C29AA2C0209303
:100400007400309375006D7D686011FB1EF4949844
:10041000959A97C09598949A94C0209162003091D3
:1004200063001091610010FB8EF44BB74F7B4BBF04
:1004300020937800309379006A7F606111FB1EF48D
:10044000C298C39A7EC0C398C29A7BC04BB74F77FD
:100450004BBF20937A0030937B00657F606211FB75
:100460001EF49498959A6DC09598949A6AC01091CC
:10047000610010FB26F418B3137F18BB62C012B3DF
:100480001F7C12BB5EC01091610010FB2EF4F09235
:10049000A000F092A10055C0F092A200F092A3003B
:1004A00050C04FC01091610010FB56F0A0EAB0E0C0
:1004B00010916200A10FBF1D109163001C9341C0F9
:1004C0001CB311FBEEF3109162001EBB1091630090
:1004D0001DBBF89414E01CBB12E01CBB789431C027
:1004E0001091610010FBFEF011FB66F0A0EAB0E095
:1004F00010916200A10FBF1DF09268001C91109333
:1005000069001FC0A0EAB0E010916200A10FBF1DFA
:100510001D912C913E91311B3323A1F7109368005C
:10052000209369000EC01CB310FBEEF31091620023
:100530001EBB11E01CBB2DB3F09268002093690034
:1005400000C07460A8950895089577FB0EF031C03F
:10055000579872FB2EF4737710919F0010680DC0AE
:10056000209170002A952093700019F573FB77771E
:100570000EF41FC010919F001F7776FB16F91093A1
:100580006600F0926F00F0926B001091660020916F
:100590006700120F20916800120F20916900120F5E
:1005A00010936A00F0926D0010916600539A1CB986
:1005B000559A579A0895089550907100552009F45E
:1005C0001DC0AEEFAD5F50906100A51918F4F09218
:1005D000710014C0F0927100EDEFF2E050906100F4
:1005E0008894551C8894EE1FFF1FE50DFF1DC895CC
:1005F000EDEFF2E0E00DFF1D09940100089508956C
:1006000064FB1EF065FBBEF00895209179003091E7
:10061000780011E0211B3F09209379003093780086
:10062000232B222341F418B3137F18BB6F7E4BB7E3
:1006300040644BBF089520917B0030917A0011E017
:10064000211B3F0920937B0030937A00232B222328
:1006500039F412B31F7C12BB6F7D4BB740644BBFA4
:020660000895FB
:00000001FF
